:100000000C945B000C947A030C94A7030C9483006B
:100010000C9483000C9483000C9483000C94830054
:100020000C9483000C9483000C9483000C94830044
:100030000C9483000C9483000C9483000C94830034
:100040000C94D4030C9483000C949E050C948300B0
:100050000C9483000C9483000C9483000C94830014
:100060000C9483000C948300000024272A000025B0
:10007000282B000023262904040404040404040299
:100080000202020202030303030303010204081035
:100090002040800102040810200102040810200002
:1000A0000000070002010000030406000000000039
:1000B00000000000960211241FBECFEFD4E0DEBF87
:1000C000CDBF11E0A0E0B1E0EEE8FCE002C0059099
:1000D0000D92AE30B107D9F711E0AEE0B1E001C04A
:1000E0001D92AE3AB107E1F710E0C6EBD0E004C0D4
:1000F0002297FE010E944106C43BD107C9F70E9426
:100100008F020C9445060C940000809102010E941D
:100110001105892B09F0ACC180911001909111015A
:10012000892B09F0A5C120E030E040EF50E060E00D
:1001300070E088E191E00E94650320E030E040E05B
:1001400050E060E070E088E191E00E94650320E00B
:1001500030E04FE050E060E070E088E191E00E9424
:10016000650320E030E040EF50E060E070E088E1BF
:1001700091E00E94650320E030E041E050E060E063
:1001800070E088E191E00E94650320E030E04FE0FC
:1001900050E060E070E088E191E00E94650381E05A
:1001A00090E0909311018093100104C0109211010E
:1001B00010921001809100010E941105892B09F015
:1001C0005FC180910E0190910F01892B09F058C1F8
:1001D00020E030E040EF50E060E070E088E191E046
:1001E0000E94650320E030E040E050E060E070E015
:1001F00088E191E00E94650320E030E040E050E0BB
:1002000060E070E088E191E00E94650320E030E06A
:1002100040EF50E060E070E088E191E00E9465030B
:1002200020E030E041E050E060E070E088E191E003
:100230000E94650320E030E040E050E060E070E0C4
:1002400088E191E00E94650381E090E090930F01C6
:1002500080930E0104C010920F0110920E01809144
:1002600004010E941105892B09F012C1809112012D
:1002700090911301892B09F00BC120E030E040EF91
:1002800050E060E070E088E191E00E94650320E0CA
:1002900030E040E050E060E070E088E191E00E94F2
:1002A000650320E030E040E050E060E070E088E18D
:1002B00091E00E94650320E030E040EF50E060E014
:1002C00070E088E191E00E94650320E030E041E0C9
:1002D00050E060E070E088E191E00E94650320E07A
:1002E00030E04FE050E060E070E088E191E00E9493
:1002F000650381E090E0909313018093120104C0A4
:100300001092130110921201809106010E941105B2
:10031000892B09F0C5C08091140190911501892B9A
:1003200009F0BEC020E030E040EF50E060E070E057
:1003300088E191E00E94650320E030E040E050E079
:1003400060E070E088E191E00E94650320E030E029
:100350004FE050E060E070E088E191E00E946503CA
:1003600020E030E040EF50E060E070E088E191E0B4
:100370000E94650320E030E041E050E060E070E082
:1003800088E191E00E94650320E030E040E050E029
:1003900060E070E088E191E00E94650381E090E018
:1003A000909315018093140104C0109215011092CE
:1003B0001401809102010E941105892B09F478C073
:1003C000809100010E941105892B09F471C0809170
:1003D00004010E941105892B09F46AC0809106016D
:1003E0000E941105892B09F463C080911601909138
:1003F0001701892B09F05CC020E030E040EF50E0AD
:1004000060E070E088E191E00E94650320E030E068
:1004100049E050E060E070E088E191E00E9465030F
:1004200020E030E040E050E060E070E088E191E002
:100430000E94650381E090E090931701809316017C
:100440000895809100010E941105892B61F080912F
:1004500004010E941105892B31F0809106010E9450
:100460001105892B61F5109217011092160108955C
:10047000809102010E941105892B09F097CE9ACE36
:10048000809100010E941105892B09F0E4CEE7CE8E
:10049000809104010E941105892B09F031CF34CFDE
:1004A000809106010E941105892B09F07ECF81CF32
:1004B000809102010E941105892BA9F2C2CF0895F3
:1004C00040E05BE460E070E088E191E00E94A1021E
:1004D00064E670E080E090E00E94440460E086E022
:1004E0000E94A80460E083E00E94A80460E085E028
:1004F0000E94A80460E084E00E94A80461E086E015
:100500000E94C60461E083E00E94C60461E085E0C9
:100510000E94C60461E084E00E94C60408950E941F
:100520006E040E9460020E948500FDCF8CE091E085
:1005300090931901809318010895862F0E949605C3
:100540000895CB01BA010E945D0508952F923F9254
:100550004F925F926F927F928F929F92AF92BF92D3
:10056000CF92DF92EF92FF920F931F93DF93CF937F
:10057000CDB7DEB7A0970FB6F894DEBF0FBECDBFE4
:100580001C016A017B01411551056105710549F4A2
:10059000DC01ED91FC910190F081E02D60E3099583
:1005A00054C0882499245401422E5524662477246B
:1005B00001E010E00C0F1D1F080D191DC701B60149
:1005C000A30192010E94EE05F80160830894811C4A
:1005D000911CA11CB11CC701B601A30192010E948C
:1005E000EE05C901DA016C017D01C114D104E104F9
:1005F000F104F1F681E0E82EF12CEC0EFD1EE80C82
:10060000F91C3E010894611C711CD501C4010197BD
:10061000A109B1096C01C818D90814C0F601EE0D82
:10062000FF1D60816A3010F4605D01C0695CD1011A
:10063000ED91FC910190F081E02DC10109950894A4
:10064000E108F1086E147F0449F7A0960FB6F894FC
:10065000DEBF0FBECDBFCF91DF911F910F91FF90F5
:10066000EF90DF90CF90BF90AF909F908F907F9052
:100670006F905F904F903F902F900895EF92FF9270
:100680000F931F93CF93DF93EC017A018B0177FFD8
:100690000FC0E881F9810190F081E02D6DE20995AC
:1006A00010950095F094E094E11CF11C011D111DC2
:1006B0002AE0B801A701CE010E94A602DF91CF91E6
:1006C0001F910F91FF90EF900895DC0121153105E6
:1006D00041F4ED91FC910190F081E02D642F09959A
:1006E00008952A30310519F40E943E0308950E94AE
:1006F000A60208951F920F920FB60F9211242F9306
:100700003F934F935F936F937F938F939F93AF9399
:10071000BF93EF93FF9380911A0190911B01892B56
:1007200029F0E0911A01F0911B010995FF91EF91D9
:10073000BF91AF919F918F917F916F915F914F91F9
:100740003F912F910F900FBE0F901F9018951F9201
:100750000F920FB60F9211242F933F934F935F93F5
:100760006F937F938F939F93AF93BF93EF93FF9379
:1007700080911C0190911D01892B29F0E0911C01B1
:10078000F0911D010995FF91EF91BF91AF919F915C
:100790008F917F916F915F914F913F912F910F902A
:1007A0000FBE0F901F9018951F920F920FB60F92C9
:1007B00011242F938F939F93AF93BF9380911E012A
:1007C00090911F01A0912001B09121010196A11DDE
:1007D000B11D80931E0190931F01A0932001B0933F
:1007E00021018091220190912301A0912401B091D7
:1007F00025018050904CAF4FBF4F809322019093C2
:100800002301A0932401B093250127C080912201E8
:1008100090912301A0912401B091250180589E431D
:10082000A040B0408093220190932301A093240123
:10083000B09325018091260190912701A091280174
:10084000B09129010196A11DB11D809326019093BD
:100850002701A0932801B093290180912201909152
:100860002301A0912401B091250181589E43A0400D
:10087000B04060F6BF91AF919F918F912F910F90F3
:100880000FBE0F901F901895EF92FF920F931F933A
:100890007B018C018FB7F89440912601509127017C
:1008A00060912801709129018FBF2FB7F894809132
:1008B000260190912701A0912801B09129012FBF15
:1008C000841B950BA60BB70BE816F9060A071B0746
:1008D00060F71F910F91FF90EF900895789484B581
:1008E000826084BD84B5816084BD85B5826085BD2C
:1008F00085B5816085BDEEE6F0E080818160808312
:10090000E1E8F0E080818260808380818160808383
:10091000E0E8F0E0808181608083E1EBF0E08081BD
:1009200084608083E0EBF0E0808181608083EAE78F
:10093000F0E0808184608083808182608083808118
:10094000816080838081806880831092C1000895D7
:10095000282F30E0C90185579F4FFC0194912958F9
:100960003F4FF9018491882381F0E82FF0E0E859A6
:10097000FF4FE491F0E0662329F48081909589236C
:10098000808308958081892B80830895482F50E0CB
:10099000CA0181569F4FFC012491CA0185579F4F80
:1009A000FC01949149585F4FFA0134913323C1F10E
:1009B000222331F1233021F4809180008F7705C00C
:1009C000243031F4809180008F7D8093800018C0A6
:1009D000213019F484B58F7704C0223021F484B516
:1009E0008F7D84BD0DC0263021F48091B0008F77BB
:1009F00005C0273029F48091B0008F7D8093B0002E
:100A0000E32FF0E0E359FF4FE491F0E0662329F48F
:100A1000808190958923808308958081892B8083AC
:100A20000895482F50E0CA0181569F4FFC01249140
:100A3000CA0185579F4FFC01949149585F4FFA01B5
:100A40003491332319F420E030E035C0222331F112
:100A5000233021F4809180008F7705C0243031F459
:100A6000809180008F7D8093800018C0213019F420
:100A700084B58F7704C0223021F484B58F7D84BD86
:100A80000DC0263021F48091B0008F7705C027304B
:100A900029F48091B0008F7D8093B000E32FF0E0C7
:100AA000EE58FF4FE491F0E0808120E030E08923B0
:100AB00011F021E030E0C9010895EF92FF920F9309
:100AC0001F937B018C0122E030E040E050E00E9467
:100AD0001006205C3D4B404F5F4FCA01B901A80191
:100AE00097010E941006C901DA010197A109B10915
:100AF000292F3A2F4B2F552747FD5A950196A11DB7
:100B0000B11D2093C50081508093C400E1ECF0E05A
:100B1000808180618083808188608083808180681B
:100B200080831F910F91FF90EF900895982F8091EF
:100B3000C00085FFFCCF9093C60008951F920F92CE
:100B40000FB60F9211242F933F934F935F936F93A0
:100B50007F938F939F93AF93BF93EF93FF934091B6
:100B6000C600E0912A01F0912B01CF01019660E8C7
:100B700070E00E94DB059C0180912C0190912D0179
:100B80002817390739F0E25DFE4F408330932B017F
:100B900020932A01FF91EF91BF91AF919F918F9187
:100BA0007F916F915F914F913F912F910F900FBE69
:100BB0000F901F90189597FB092E07260AD077FDF6
:100BC00004D049D006D000201AF4709561957F4F6B
:100BD0000895F6F7909581959F4F0895A1E21A2EFA
:100BE000AA1BBB1BFD010DC0AA1FBB1FEE1FFF1FD1
:100BF000A217B307E407F50720F0A21BB30BE40B21
:100C0000F50B661F771F881F991F1A9469F7609567
:100C10007095809590959B01AC01BD01CF01089521
:100C200097FB092E05260ED057FD04D0D7DF0AD03A
:100C3000001C38F450954095309521953F4F4F4F0B
:100C40005F4F0895F6F790958095709561957F4F69
:100C50008F4F9F4F0895AA1BBB1B51E107C0AA1FCE
:100C6000BB1FA617B70710F0A61BB70B881F991F4D
:100C70005A95A9F780959095BC01CD010895EE0F86
:0E0C8000FF1F0590F491E02D0994F894FFCF2A
:0E0C8E000600030005000400000000009D02A7
:00000001FF
